:1000000017C1000031C100002FC100002DC1000048
:100010002BC1000029C1000027C1000025C100003C
:1000200023C1000021C100001FC100000C94F10891
:100030000C94B80819C1000017C1000015C10000D8
:1000400013C1000011C100000FC100000DC100006C
:100050000BC1000009C1000007C1000005C100007C
:1000600003C1000001C10000FFC00000FDC000008E
:10007000FBC000004D542D44422D55312044656D88
:100080006F2050726F6772616D004669726D7761A3
:100090007265205265766973696F6E203131303533
:1000A000303900687474703A2F2F7777772E6D612E
:1000B0007474616972746563682E636F6D2F004D8F
:1000C000542D44422D55312044656D6F004C4544FC
:1000D0000A43726564697473004C45442069732057
:1000E0006E6F7720666C617368696E67004A75731E
:1000F00074696E204D6174746169720A4465616E41
:100100002043616D657261202D204C55464120557C
:100110005342206C6962726172790A41746D656C38
:1001200020436F72706F726174696F6E0044656D09
:100130006F20686173206E6F74206265656E207732
:1001400072697474656E0A436865636B20776562D3
:100150007369746520736F6F6E21001201100102C4
:10016000000010D016570501000102000109023EEF
:1001700000020100C0640904000001020201000540
:10018000240010010424020605240600010705824C
:10019000030800FF09040100020A0000000705042B
:1001A0000220000107058302200001040309042046
:1001B000034D006100740074006100690072005416
:1001C0000065006300680020004C004C0043000004
:1001D000001C034D0054002D00440042002D00552A
:1001E0000031002000440065006D006F0000000E2B
:1001F0000331003100300035003100300000005084
:100200007265737320616E79206B6579004E657736
:10021000206865782076616C75653A004261636B91
:1002200000204F4B20002043414E43454C2000000E
:1002300011241FBECFEFD2E0DEBFCDBF11E0A0E0A2
:10024000B1E0E4E5F8E102C005900D92A830B107F5
:10025000D9F711E0A8E0B1E001C01D92AB39B107B8
:10026000E1F71ED10C94280CCBCE84E08093E900FA
:100270008091F200811181E0089584EC99E028ECEE
:1002800030E0F9013197F1F70197D9F782E008954D
:1002900083B7817F83BF589A08955898789483B71D
:1002A000817F846083BF83B7816083BF889583B774
:1002B0008E7F83BF0895089580919401813229F043
:1002C000823259F1803299F513C080919301813ABD
:1002D00071F58091E800877F8093E80080E091E0ED
:1002E00067E070E00E94DD0A8091E8008B7712C021
:1002F000809193018132D9F48091E800877F8093C7
:10030000E80080E091E067E070E00E94390B8091A6
:10031000E8008E778093E800089580919301813200
:1003200031F48091E800877F8093E800BBC6089590
:10033000589A82E061EC42E080D6882339F083E06D
:1003400061E846E27AD6882351F002C05898F7CF88
:1003500084E060E846E271D6882319F003C058981B
:10036000F7CF5898109200011092010110920201EB
:1003700010920301089581E061E01DD28AE260E5F8
:100380002DD182E06DE117D284E790E0FCD183E0CB
:100390006CE111D28AE890E0F6D184E06AE10BD2F8
:1003A00083EA90E0F0D185E061E005D28AE260E581
:1003B00015C11F93CF93DF93EC0111E01CC0809116
:1003C0000A018823C1F0AA9B16C0AA9A809108014D
:1003D000882331F088B58F3F41F41092080108C09E
:1003E00088B5882329F41093080188B58F5F02C06F
:1003F00088B5815088BDCE0160E0F1D58823F9F23F
:1004000080E0DF91CF911F910895ACC50895CFC5CD
:10041000089584B7877F84BF88E10FB6F8948093EE
:100420006000109260000FBE91E080E80FB6F89473
:1004300080936100909361000FBE83B7817F83BF7B
:100440005898509A57985F9A84D6789408950F9345
:100450008DEE90E06DEC70E043E024E001E07CD4B0
:100460000F9108950F9383E284BD8FEF88BD1092A2
:10047000080183E085BD81E080930A0189ED90E069
:100480006DEC70E040E024E001E066D48130B1F72B
:1004900010920A0114BC15BCAA9A589A0F9108959B
:1004A0000F93B7DF3ED58DEC90E06FEB70E040E04E
:1004B00020E001E051D4813011F4D4DFF4CFC7DF64
:1004C000F2CFDA01923049F0933061F0913029F5A2
:1004D000EBE5F1E022E130E024C0EDE6F1E02EE3CF
:1004E00030E01FC0813059F0813028F0823059F05F
:1004F000833099F40CC0EBEAF1E084910BC0EFEA91
:10050000F1E0849107C0E1EDF1E0849103C0EFEEEA
:10051000F1E08491282F30E004C0E0E0F0E020E03A
:1005200030E0ED93FC93C90108950F931F93DF937F
:10053000CF930F92CDB7DEB719828E010F5F1F4F99
:10054000C80137DF282F30E02130310511F439811F
:100550001BC080918D01813091F0813018F0823084
:1005600071F51EC089818B3119F0282F30E027C02A
:1005700081E080938D01C8011CDF282F30E0998134
:100580002130310519F4392F20E019C09B3599F439
:1005900082E080938D01CE0101960BDF282F30E0A1
:1005A00099812130310579F3892F8154843018F4F1
:1005B000392F20E002C0292F30E010928D01C901AF
:1005C0000F90CF91DF911F910F910895982F8091F7
:1005D0000701882311F0892F1ACF0895FF920F93F6
:1005E0001F93F82E062F10E003C08F2DEFDF1F5F43
:1005F0001017D8F31F910F91FF9008951F93182F94
:100600008BE1E4DF8BE5E2DF812FE0DF8DE6DEDFEB
:100610001F9108958BE1DADF8BE5D8DF82E3D6DF27
:100620008AE4D4CF2F923F924F925F926F927F9243
:100630008F929F92AF92BF92CF92DF92EF92FF92F2
:100640000F931F93DF93CF9300D0CDB7DEB79A837C
:100650008983842E9924EE24FF24F394C62EDD246E
:1006600043E0A42EB12CAC20BD201E010894211C17
:10067000311C34E0432E512C4C205D2020E1622EB1
:10068000712C6C207D20A114B10441F4E981FA8120
:100690003196FA83E983319784913CC009811A81AC
:1006A00081E0A816B10491F5C1010E94200C29C077
:1006B0008E1499F44114510479F46114710451F0C9
:1006C000E0910B01F0910C01F192F0930C01E09399
:1006D0000B0102C08F2D7ADF9394A114B10441F471
:1006E000E981FA813196FA83E9833197849112C0C6
:1006F00009811A8181E0A816B10441F4C1010E9468
:10070000200C0F5F1F4F1A83098304C0F8018191E9
:10071000FA83E9839F2DF82E8AE0F81611F0FF2066
:1007200039F6E394FF2009F0AECFC4FE0AC0E09191
:100730000B01F0910C018AE08193F0930C01E0939E
:100740000B01C3FC02C0E92C03C09A3009F4EA94FF
:100750008E2D0F900F90CF91DF911F910F91FF90F1
:10076000EF90DF90CF90BF90AF909F908F907F9051
:100770006F905F904F903F902F900895482F8DE09D
:1007800091E062E04FCF60E040E04CCF1F93182F24
:1007900080E302C08F5F14561436E0F717DF80E362
:1007A00002C08F5F1A501A30E0F710DF812F805D92
:1007B0000DDF1F9108950F931F93182F062F8BE1C4
:1007C00005DF8BE503DF812FE1DF8BE3FFDE802F89
:1007D000DDDF88E4FBDE1F910F91089586E061E084
:1007E000EACFBF92CF92DF92EF92FF920F931F93C7
:1007F000CF93DF93E82E062FD42E122FC62ECA9445
:10080000D3941D5F6C2DD7DF8BE2E0DEB12EBC0CE4
:100810008E2D6B2DD0DF8BE2D9DEFD2CFE0C8F2DC3
:100820006C2DC9DF8AE2D2DE8F2D6B2DC4DF8AE208
:10083000CDDECC2DD0E0C10FD11D1E2D1E5F10C00E
:100840008E2D602FB8DF8DE2C1DE812F602FB3DFE8
:100850008DE2BCDE8F2D602FAEDF8DE2B7DE0F5F45
:10086000802F90E08C179D075CF3FE2CF3940E2DE7
:1008700010E00D0D111D0BC08F2D6C2D9CDF8CE732
:10088000A5DE8F2D6B2D97DF8CE7A0DEF3948F2DE7
:1008900090E08017910784F3DF91CF911F910F9122
:1008A000FF90EF90DF90CF90BF9008952F923F92EE
:1008B0004F925F926F927F928F929F92AF92BF9270
:1008C000CF92DF92EF92FF920F931F93DF93CF931C
:1008D000CDB7DEB7A9970FB6F894DEBF0FBECDBF78
:1008E000988B8F877A8B698B4B8B122FEC8A2170B8
:1008F0002C83009719F02E839C0104C032E03E83C4
:100900002DE031E0C12EDD24C60144E096958795A7
:100910004A95E1F796E0892E882246E0841611F484
:10092000B8E08B2E6E816C60C90140E07BDEA2E0F6
:100930004A2E480E960120713070F601E470F07076
:10094000FE87ED87C2FE14C0232B11F023E006C002
:10095000212F2095221F2227221F220F882019F0E5
:10096000F3E0F88703C0342D3E5F3887420E0AC09B
:10097000232B19F443E0488705C0F3E04F2E480EBF
:1009800053E0588710920701C601807190709B83D5
:100990008A83E4E095958795EA95E1F7EDEFE81B0A
:1009A000EC87242D30E0C901029662E070E021D787
:1009B000709561957F4FF62FF45FF9831D8299241E
:1009C0001B8641E04A8749874F83C90102979B8F65
:1009D0008A8FF9013197FD8FEC8FF8858F2F90E08A
:1009E000602E77249C01260D371D3F8F2E8F089493
:1009F00061087108A301480F591F59A348A308941F
:100A0000611C711CF601E270F070FBA3EAA39C016B
:100A1000215030403DA32CA3A601447150705FA328
:100A20004EA360C18F859889009711F01C0106C004
:100A300092E09E837DE0272E71E0372E5524E985D4
:100A4000EF5FED8B3F81232F30E03F8B2E8B49856D
:100A50004150488F59855350598F19C15394852D52
:100A600090E0882031F4E8A1F9A18E179F07B9F42E
:100A700014C02A8D3B8D821793072CF448A159A1ED
:100A80008417950751F0EC8DFD8D8E179F073CF074
:100A90002E8D3F8D8217930711F487E301C080E309
:100AA000ADDD1A85150D812F6D8985DE31E0531678
:100AB000B9F44D81941610F460E006C05D8156953E
:100AC000692D66956F5F651B8985680F812F73DEC1
:100AD00089899A896C814B89A5DDE82E8D836EC04A
:100AE00092E0591609F469C0E3E05E16E9F42A8140
:100AF0003B81232B09F425C14D855E85452B09F0EB
:100B000020C18CE192E03FDEE82E10E0C92CDD240C
:100B1000C81AD10803C080E259DD1F5F812F90E021
:100B20008C159D05C4F34AC0852D90E0ECA1FDA174
:100B30008E179F0739F42D853E85232B19F08820C9
:100B400019F43BC0882029F04A8D5B8D84179507E6
:100B5000A1F15885551639F4ED85FE85EF2B19F076
:100B6000882041F002C08820A9F02C8D3D8D82178D
:100B7000930781F4692D66954A815B81452B39F095
:100B8000598D650F812F17DE86E292E013C0888DA4
:100B9000680F0CC0541409F0D4C0EEA1FFA17497E3
:100BA00009F0CFC0692D6695F88D6F0F812F03DE98
:100BB00081E292E0E8DDE82E01C0EE2400E060C0B2
:100BC000882011F080E31ADD10E0CE88DF88CE188F
:100BD000D10803C080E2FADC1F5F812F90E08C1502
:100BE0009D05C4F38820A1F1252D30E039A728A761
:100BF000C9010397682D70E0EAD56DE0C62E61E06B
:100C0000D62EC80ED91E10E05EEFA52E5FEFB52ED2
:100C1000A20EB31E3C89311729F46A147B0411F427
:100C200085E301C080E3EADCF60181916F01CEDC4F
:100C30001F5F181578F328A539A522503040621699
:100C4000730611F487E301C080E3D8DC082D04C0EB
:100C50008C85850D93DD082FF92C3F81F31AF01A4E
:100C600003C0F92CFE1800E010E003C080E2AEDC07
:100C70001F5F1F15D8F38E2D90E00196280E391EA8
:100C80009E1408F49E2C4B85401708F40B875414CF
:100C900008F4E4CE5981573018F487E08A8702C0FF
:100CA00099819A87EAA1FBA1EF2B59F0F92DFC5FFE
:100CB000FF8380910701882321F42B85920E34E075
:100CC000930E892D90E0049662E070E092D57095C5
:100CD00061957F4F462F485D4987809107018F5F5F
:100CE0008093070180910701823008F49BCE80E356
:100CF00085DC8A856985442D292D73DD6FDD88208B
:100D000019F0842D835004C0842D8F5F5885851B76
:100D1000A9960FB6F894DEBF0FBECDBFCF91DF917D
:100D20001F910F91FF90EF90DF90CF90BF90AF9009
:100D30009F908F907F906F905F904F903F902F90FB
:100D40000895C1016E8140E06DDCE82E8AA19BA16F
:100D5000892B09F035CF85CF2F923F924F925F922A
:100D60006F927F928F929F92AF92BF92CF92DF92BB
:100D7000EF92FF920F931F93DF93CF9300D00F92C8
:100D8000CDB7DEB71C012B014983C22E102F30E0F6
:100D9000C901807690709B838A8374E096958795CD
:100DA0007A95E1F7D82E96E0D91611F468E0D62EA0
:100DB000FF246D2C7724430108948108910858E0A2
:100DC000A52EB12CA222B32201C0102F23DCD3DA2E
:100DD000C101B20149812C2D012FEF2C67DD082FB5
:100DE00014DBC7FE03C010928E0137C09EDBDC010E
:100DF0008D30910581F4EA81FB81EF2B41F0802F4A
:100E000090E00197212F30E028173907A4F18DE0F9
:100E100080938E016FC0882371F5B0938E01B13439
:100E200031F4115099F6A114B10479F262C0B234D0
:100E300051F41F5F011750F6A114B10411F0102FE7
:100E400059C011E0C3CFB43431F48A819B81892B1E
:100E500009F04AC04FC0B33411F010E04BC0EA8132
:100E6000FB81EF2B09F446C08F2D90E08815990582
:100E70000CF0ACCF34C08A819B81892B09F4A6CFBA
:100E8000412F50E0802F90E00197481759070CF050
:100E90009DCFFD1430F5CD01C0970A9750F0CD01DC
:100EA00081549040069728F0CD01815690400697D6
:100EB000C0F4CD0181569040069708F490972F2DED
:100EC00030E0CA010197B30182D4F901E35FFE4F1C
:100ED000E80FF91FA083281539050CF077CFF3949C
:100EE00075CF189709F072CFFF2009F46FCFFA94ED
:100EF0006DCF11E0812F0F900F900F90CF91DF9168
:100F00001F910F91FF90EF90DF90CF90BF90AF9027
:100F10009F908F907F906F905F904F903F902F9019
:100F20000895DF93CF930F92CDB7DEB773DB23DA4B
:100F30008CE061E240DC8FEF91E025DC4FDC65DA8C
:100F400094D9882339F0CE01019633DA813029F023
:100F500082E004C092D9813049F780E00F90CF91B0
:100F6000DF9108951F931091E90083E08093E900D9
:100F70009091E8008091E8008E778093E80095FFDB
:100F800002C00CC012D48091E80080FFFBCF80919A
:100F9000E8008E778093E80001C007D48091E800D4
:100FA00080FFFBCF17701093E9001F9108951F93E6
:100FB000182F83E08093E9008091E80085FD0BC045
:100FC0008091E8008E778093E80001C0EED3809195
:100FD000E80080FFFBCF1093F1001F910895CF939D
:100FE000DF93EC0184E08093E900662381F0809137
:100FF000F2008823A1F48091E8008B778093E800C9
:1010000001C0D3D38091E80082FDF1CFFACF809167
:10101000E80082FF0EC08091F200882329F08091C1
:10102000F100888381E006C08091E8008B7780938F
:10103000E80080E0DF91CF910895382F282F2CC051
:101040002093E900231721F4762F942F50E006C057
:101050007091EC009091ED005091F00091FF1BC059
:101060008091EB008E7F8093EB008091ED00827089
:101070008093ED008091EB0081608093EB00709392
:10108000EC009093ED005093F0008091EE0087FD0E
:1010900002C080E008952F5F253090F23093E90080
:1010A00081E008958091930188238CF403C08EB36E
:1010B0008823B1F08091E80082FFF9CF8091E800A9
:1010C0008B778093E80008958EB3882349F0809150
:1010D000E80080FFF9CF8091E8008E778093E800E8
:1010E000089540D042D08091D800982F9F77909358
:1010F000D80080688093D8008091D8008F7D80933D
:10110000D80084E089BD89B5826089BD09B400FE3C
:10111000FDCF1EBA109291011092900110928F0192
:1011200080E060E042E189DF8091E1008E7F809382
:10113000E1008091E20081608093E2008091E20012
:1011400088608093E2008091E0008E7F8093E000D1
:101150000895E3E6F0E080818E7F808381E08093D4
:101160009201BFCF1092E20008951092E10008951D
:101170001F920F920FB60F9211241F932F933F933C
:101180004F935F936F937F938F939F93AF93BF938F
:10119000EF93FF93E9EEF0E0108117701082E0EF1B
:1011A000F0E08081877F80837894C2D0A9EEB0E0A0
:1011B0001C92E0EFF0E08081886080831C93FF91B7
:1011C000EF91BF91AF919F918F917F916F915F91BF
:1011D0004F913F912F911F910F900FBE0F901F9035
:1011E00018951F920F920FB60F9211242F933F93D1
:1011F0004F935F936F937F938F939F93AF93BF931F
:10120000EF93FF938091E10082FF0AC08091E2009A
:1012100082FF06C08091E1008B7F8093E100CCD1FA
:101220008091E10080FF16C08091E20080FF12C033
:101230008091E2008E7F8093E2008091E2008061E5
:101240008093E2008091D80080628093D80019BC1E
:101250001EBA23D88091E10084FF2EC08091E20065
:1012600084FF2AC084E089BD89B5826089BD09B444
:1012700000FEFDCF8091D8008F7D8093D8008091B3
:10128000E1008F7E8093E1008091E2008F7E809369
:10129000E2008091E20081608093E2008091910100
:1012A000882331F48091E30087FD02C081E001C012
:1012B00084E08EBB0E9448018091E10083FF27C03B
:1012C0008091E20083FF23C08091E100877F8093BB
:1012D000E10082E08EBB109291018091E1008E7F4F
:1012E0008093E1008091E2008E7F8093E200809104
:1012F000E20080618093E20080E060E042E19DDEF8
:101300008091F00088608093F0000E945B01FF9163
:10131000EF91BF91AF919F918F917F916F915F916D
:101320004F913F912F910F900FBE0F901F901895E6
:101330000F931F93DF93CF9300D0CDB7DEB780918B
:10134000F100809393018091F1008093940180914A
:10135000F1009091F100E5E9F1E08093950190931F
:1013600096018091F1009091F10080939701938311
:101370008091F1009091F1008093990195830E94F2
:101380005C018091E80083FF02C18091930130915C
:101390009401353009F487C0363040F43130C9F15A
:1013A000313070F0333009F0F2C033C0383009F416
:1013B000C0C0393009F4CFC0363009F0E8C098C059
:1013C000803821F0823809F0E2C008C090918F0186
:1013D00080919001882399F0926011C080919701CB
:1013E00087708093E9008091EB0090E025E096956E
:1013F00087952A95E1F7982F91701092E9008091D6
:10140000E800877F8093E8009093F1001092F1004C
:101410009BC0882319F0823009F0B9C090E08F7129
:101420009070009721F0029709F0B1C00CC0809134
:101430009501813009F0ABC010929001333069F50D
:10144000809390012AC080919501882331F52091E5
:101450009701277009F49BC02093E9008091EB006D
:1014600080FF1BC0333021F48091EB00806213C0F9
:101470008091EB0080618093EB0081E090E002C0FE
:10148000880F991F2A95E2F78093EA001092EA00EC
:101490008091EB0088608093EB001092E9008091CE
:1014A000E800877F54C0882309F071C0109195012E
:1014B0001F770FB7F8948091E800877F8093E8004A
:1014C000F1DD8091E80080FFFCCF8091E30080781F
:1014D000812B8093E3008091E30080688093E30098
:1014E000112311F482E001C083E08EBB0FBF4FC017
:1014F0008058823008F04BC0809195019091960100
:1015000060919701AE014F5F5F4F0E946102BC0185
:10151000009709F43CC08091E800877F8093E80041
:1015200089819A81E3D08091E8008B778093E800ED
:101530002EC0803861F58091E800877F8093E800B5
:10154000809191018093F1008091E8008E778093E3
:10155000E800A8DD1CC08823D1F490919501923059
:10156000B0F48091E800877F8093E8009093910128
:1015700099DD80919101882331F48091E30087FD0A
:1015800002C081E001C084E08EBB0E94980180917E
:10159000E80083FF0AC08091EB0080628093EB003B
:1015A0008091E800877F8093E8000F900F90CF91A3
:1015B000DF911F910F91089508959C014091990129
:1015C00050919A014617570718F4F90190E03CC072
:1015D0006115710511F0AB01F8CF8091E8008E77AD
:1015E0008093E80040E050E0F0CF8EB38823E9F12B
:1015F0008530E9F18091E80083FF02C081E0089521
:101600008091E80082FD2BC08091E80080FF1CC023
:101610008091F200282F30E007C081918093F10083
:10162000415050402F5F3F4F4115510519F0203177
:10163000310598F390E02031310509F491E0809173
:10164000E8008E778093E8004115510571F69923E3
:1016500061F605C08EB3882341F0853041F080915A
:10166000E80082FFF7CF80E0089582E0089583E0EC
:1016700008959C016115710529F48091E8008B772C
:101680008093E800F9011FC08EB3882359F185309B
:1016900059F18091E80083FF02C081E008958091B4
:1016A000E80082FFF1CF06C08091F1008193615084
:1016B000704021F08091F2008823B1F78091E8001A
:1016C0008B778093E80061157105F1F605C08EB344
:1016D000882341F0853041F08091E80080FFF7CF0A
:1016E00080E0089582E0089583E008959C01409190
:1016F000990150919A014617570718F4F90190E0A3
:101700003FC06115710511F0AB01F8CF8091E80081
:101710008E778093E80040E050E0F0CF8EB38823CE
:1017200009F43FC0853009F43EC08091E80083FF92
:1017300002C081E008958091E80082FD2CC0809174
:10174000E80080FF1DC08091F200282F30E008C023
:1017500084918093F1003196415050402F5F3F4F6C
:101760004115510519F02031310590F390E02031F9
:10177000310509F491E08091E8008E778093E800CC
:101780004115510559F6992349F605C08EB38823B2
:1017900041F0853041F08091E80082FFF7CF80E092
:1017A000089582E0089583E008951F938EB38823FF
:1017B00061F01091E9001092E9008091E80083FF48
:1017C00001C0B6DD17701093E9001F9108955527E9
:1017D000002480FF02C0060E571F660F771F611599
:1017E000710521F096958795009799F7952F802D93
:1017F000089597FB092E07260AD077FD04D00CD058
:1018000006D000201AF4709561957F4F0895F6F781
:10181000909581959F4F0895AA1BBB1B51E107C06E
:10182000AA1FBB1FA617B70710F0A61BB70B881F70
:10183000991F5A95A9F780959095BC01CD010895FF
:10184000F999FECF92BD81BDF89A992780B5089588
:04185000F894FFCF3A
:08185400000000000000080183
:00000001FF
